:100000000C94DA030C94F7030C94F7030C94F703A5
:100010000C94F7030C94F7030C94F7030C94F70378
:100020000C94F7030C94F7030C947B2D0C944D2E39
:100030000C94B1230C94F7030C94F7030C94F7037E
:100040000C94F7030C94F7030C94F7030C94F70348
:100050000C94F7030C9419240C94F7030C94F703F5
:100060000C94F7030C94F7030C94F7030C94F70328
:100070000C94F7030C94F7030C94F7030C94F70318
:100080000C94F7030C94F7030C94F7030C94F70308
:100090000C94F7030C94F7030C94F7030C94F703F8
:1000A0000C94F7030C94F7030C94F7034F045204D9
:1000B000550458045B045D046004A007A507AF075E
:1000C000A307A807AD07AB07E808EA08F508EC089E
:1000D000EE08F008F208F408F708F908FB0806092A
:1000E000FD08FF080109030905090809111911197B
:1000F000431943197A199A19031B611BDC19611BF7
:10010000891A891AFA1A611B611B5B1B961A961AC7
:10011000961A961A961A961A961A961A961A961A5F
:10012000961A961A961A961A961A961AA71AB41A20
:10013000BB1AC21ACC1AEC1BEC1BFE1BFE1BF51BD8
:10014000FE1BFE1BFE1BEC1BEC1BFA1BFE1BFE1B0F
:10015000FA1BBA2EE12ED32FE12ED32F2D2F502FA5
:10016000D32FA62FB52F07634236B79BD8A71A39CE
:10017000685618AEBAAB558C1D3CB7CC5763BD6DF5
:10018000EDFD753EF6177231BF000000803F05A8F7
:100190004CCDB2D44EB93836A9020C50B9918688EC
:1001A000083CA6AAAA2ABE000000803F6572676FBD
:1001B000646F785F657A2F3864353131363736664B
:1001C0006135316332373738303862204020302E85
:1001D000362E3133382D392D673330326537322D95
:1001E0006469727479000000F0A135022B003900B7
:1001F000E100E00000001E00140004001D00E30008
:1002000029001F001A0016001B00E2002A0020002F
:100210000800070006001E082C0021001500090038
:1002200019001F084A00220017000A0005000000FC
:1002300009042D00015100002F00000035002D029F
:100240000251000030000000E20023001C000B00FF
:10025000110000002804240018000D0010002E00DA
:100260004B0025000C000E0036002D002C0026004F
:1002700012000F00370034022A0027001300330059
:100280003800280428002A0031003400E500015419
:1002900000000100010001000100010000001E0833
:1002A000F400F2000100010001001F08F000F1005D
:1002B0000100010001002008F500F3000100010029
:1002C00001002108010001000100010001002208D5
:1002D0000100010001000000010001000100000018
:1002E0000100000001000100010000000100000009
:1002F0000100230801005000010000000100240853
:100300000100510001000100010025080100520018
:10031000010001000100260801004F00010001005A
:100320000100270801000100010001000100010097
:1003300001000100010001000000010001000100B6
:100340000100010000003A0001000100010001006D
:1003500001003B00010001000100010001003C0020
:10036000010001000100010001003D000100010049
:100370000100010001003E00010001000100000039
:10038000010001001901000013010000010001003B
:10039000010000000100000001003F000100010019
:1003A0000100000001004000010001000100010007
:1003B00001004100010001000100010001004200B4
:1003C00001000100010001000100430001000100E3
:1003D000010001000100440045004C000100010043
:1003E000000000000000000000002A2B2800000090
:1003F00000000000000000000000000000290000D4
:1004000000002C1E3420212224342627252E362DB0
:100410003738271E1F202122232425263333362E4A
:1004200037381F0405060708090A0B0C0D0E0F10BC
:100430001112131415161718191A1B1C1D2F313001
:10044000232D350405060708090A0B0C0D0E0F10A5
:100450001112131415161718191A1B1C1D2F3130E1
:10046000354C00000000000000000000000000000B
:10047000000000000000000000000000000000007C
:100480000000000101010101010001010101000062
:10049000000000000000000000000000010001005A
:1004A000010101010101010101010101010101013C
:1004B000010101010101010101010101010000002F
:1004C000010100000000000000000000000000002A
:1004D0000000000000000000000000000001010119
:1004E000010000047F3F1F643214643214783C1E04
:1004F0001E140A056801F000B40078005A000000DC
:1005000000000001010101010101010102020202DA
:1005100002020202020303030303030303040404AD
:100520000404040505050505060606060607070773
:1005300007080808080909090A0A0A0A0B0B0B0C24
:100540000C0C0D0D0D0E0E0F0F0F101011111112BE
:100550001213131414151516161717181819191A3B
:100560001A1B1C1C1D1D1E1F1F202021222223249C
:10057000252526272728292A2B2B2C2D2E2F2F30D7
:10058000313233343536363738393A3B3C3D3E3FED
:100590004041424344464748494A4B4C4D4F5051D5
:1005A0005253555657585A5B5C5E5F60626364668F
:1005B00067696A6C6D6E707173747678797B7C7E16
:1005C0008081838486888A8B8D8F91929496989A65
:1005D0009B9D9FA1A3A5A7A9ABADAFB1B3B5B7B97B
:1005E000BBBDBFC1C4C6C8CACCCFD1D3D6D8DADC54
:1005F000DFE1E4E6E8EBEDF0F2F5F7FAFCFF0403E7
:100600003000000016034500720067006F004400D0
:100610006F007800200045005A00000016034500D6
:10062000720067006F0044006F00780020004500F2
:100630005A0000000403090409026D00040100A02F
:10064000FA09040000010301010009211101000160
:100650002240000705810308000A09040100010384
:10066000010200092111010001224D00070582034A
:1006700008000A0904020001030000000921110119
:1006800000012236000705830308000A090403005D
:1006900001030000000921110100012239000705B2
:1006A00084032000011201100100000008EDFE0784
:1006B0001301000102030105010906A10105071943
:1006C000E029E71500250195087501810205081943
:1006D00001290595057501910295017503910105A3
:1006E00007190029F71500250195F875018102C049
:1006F00005010980A10185021601002603001A8167
:10070000002A8300751095018100C0050C0901A124
:10071000018503160100269C021A01002A9C02751D
:100720001095018100C005010902A1010901A10084
:100730000509190129051500250195057501810295
:100740009501750381010501093009311581257F66
:1007500095027508810609381581257F9501750870
:100760008106050C0A38021581257F9501750881DF
:1007700006C0C005010906A101050719E029E71512
:100780000025019508750181029501750881010513
:1007900008190129059505750191029501750391C7
:1007A000010507190029FF150026FF0095067508A9
:1007B0008100C00011241FBECFEFDAE0DEBFCDBF45
:1007C00011E0A0E0B1E0EAEAF7E602C005900D9280
:1007D000A83EB107D9F723E0A8EEB1E001C01D9211
:1007E000AD3BB207E1F70E94A02A0C94D3330C94DE
:1007F000000080B38C7080BB81B3836F81BB089590
:1008000084B1807F84B985B1807F85B98AB1837FC7
:100810008AB98BB1837F8BB93E9846980895CF9360
:10082000E82F873090F58091000190910101892B8C
:1008300009F048C0CE2F64E670E080E40E94A6056F
:100840009093010180930001892BD1F464E670E05C
:1008500082E10E94FD059093010180930001892BA4
:1008600079F481E090E001C0880FCA95EAF764E668
:1008700070E080950E94FD05909301018093000136
:1008800084E690E0CF910C94520690E0FC013797FB
:10089000E730F105B8F4EA5AFF4F0C947833209A08
:1008A000289810C0219A29980DC0229A2A980AC027
:1008B000239A2B9807C0529A01C0539A5B9802C0A2
:1008C0003E9A4698CF910895CF93873008F041C063
:1008D0008091000190910101892B09F043C064E6E9
:1008E00070E080E40E94A6059093010180930001CE
:1008F000892B11F0C0E027C064E670E083E10E941C
:10090000FD059093010180930001892B99F764E61E
:1009100070E081E40E94A60590930101809300019C
:10092000892B41F784E690E00E942D0697FF05C0D1
:100930009093010180930001DDCFC82FC0951092E4
:1009400001011092000184E690E00E9452068C2F73
:100950000AC09FB18FB1807F869586959370892B51
:10096000809501C080E0CF910895089508950C947A
:10097000B6040E94E40690E0909301018093000188
:100980000E9400040E94F90329EE31E0EDE3F2E059
:100990004EE04E0F119280E090E0D901A80FB91FF0
:1009A0001C92019686309105C1F72A5F3F4F4E1386
:1009B000F1CF0C9418080E94E40690E09093010196
:1009C000809300010E9400040E94F903EDE3F2E02D
:1009D0008EE08E0F11928E13FDCF089526E0829F38
:1009E000C0011124FC01E751FE4F20E030E080E01F
:1009F00041E050E09081992319F09150908307C015
:100A0000BA01022E01C0660F0A94EAF7862B2F5F07
:100A10003F4F31962630310569F7089596E0699F7A
:100A2000B001112420E030E090E04FE0FC01022E04
:100A300002C0F595E7950A94E2F7E0FF06C0F901D8
:100A4000E60FF71FE751FE4F40832F5F3F4F2630E1
:100A5000310561F70895CF92DF92EF92FF920F93E5
:100A60001F93CF93DF938091000190910101892B17
:100A700091F08091E8018F5F8093E80181110BC0B4
:100A80000E94E40690E09093010180930001892B7D
:100A900011F40E9476068DE3C82E82E0D82E94E4ED
:100AA000E92E92E0F92EC0E08C2F0E940F0407E09F
:100AB0000C0F802F0E940F048C2F0E94EE04182F21
:100AC0008C2F0E946404F6019081D12FD095D923F8
:100AD0008123D82B6C2F8D2F89270E940E05F601BC
:100AE000D1936F01802F0E94EE04182F802F0E9457
:100AF0006404F7019081D12FD095D9238123D82B7D
:100B0000602F8D2F89270E940E05F701D1937F0159
:100B10000E940004CF5FC73039F60E94240881E0AC
:100B2000DF91CF911F910F91FF90EF90DF90CF90C9
:100B30000895E82FF0E0E35CFD4F8081089508956B
:100B40001092B9008CE08093B8000895EF92FF9264
:100B50000F931F93CF93DF93182FEB011092BC00DC
:100B600084EA8093BC000E94E3237C019091BC0046
:100B700097FD0EC0CF3F8FEFD807C1F30E94E3234C
:100B80008E199F098C179D0788F38EEF9FEF2EC05B
:100B90009091B900987F983041F09091B900987F7A
:100BA000903119F08FEF9FEF21C01093BB0084E8C4
:100BB0008093BC000E94E3238C019091BC0097FDC0
:100BC0000CC0CF3F8FEFD807C1F30E94E323801BF7
:100BD000910B8C179D0788F3D8CF8091B900887F3F
:100BE000883111F08034F1F680E090E0DF91CF9110
:100BF0001F910F91FF90EF9008950F931F93CF9344
:100C0000DF93EB018093BB0084E88093BC000E94DB
:100C1000E3238C019091BC0097FD0EC0CF3F8FEF76
:100C2000D807C1F30E94E323801B910B8C179D070B
:100C300088F38EEF9FEF0CC02091B900287F81E0F0
:100C400090E0283211F480E090E09195819591092F
:100C5000DF91CF911F910F9108950F931F93CF9321
:100C6000DF93EC0184E88093BC000E94E3238C01B5
:100C70009091BC0097FD0EC0CF3F8FEFD807C1F316
:100C80000E94E323801B910B8C179D0788F38EEF46
:100C90009FEF03C08091BB0090E0DF91CF911F9147
:100CA0000F9108950F931F93CF93DF93EC0184E985
:100CB0008093BC000E94E3238C019091BC0094FFC0
:100CC0000EC0CF3F8FEFD807C1F30E94E323801BF4
:100CD000910B8C179D0788F38EEF9FEF02C080E089
:100CE00090E0DF91CF911F910F91089556985E98F3
:100CF00025982D9826982E9827982F988FEF90E07A
:100D0000909389008093880090938B0080938A0051
:100D100090938D0080938C00259A2D9A2FEF80E779
:100D200092E0215080409040E1F700C00000269AF8
:100D30002E9A2FEF80E792E0215080409040E1F71B
:100D400000C00000279A2F9A2FEF80E792E02150F1
:100D500080409040E1F700C0000025982D982FEFCB
:100D600080E792E0215080409040E1F700C0000011
:100D700026982E982FEF80E792E0215080409040F7
:100D8000E1F700C0000027982F9856985E982598A4
:100D90002D9826982E9827982F98089589EA809361
:100DA000800089E08093810024982C983F988AB134
:100DB0008F7C8AB96E98479A8BB180638BB9769A8B
:100DC0000E9476060C94B50480E290E090930101B5
:100DD0008093000180914B0281110EC00E94A005FA
:100DE00081E080934B022FEF83ED90E32150804010
:100DF0009040E1F700C0000064E670E080E40E94EB
:100E0000A6059093010180930001892B09F050C041
:100E100064E670E080E00E94FD05909301018093FC
:100E20000001892B09F044C064E670E080E00E9474
:100E3000FD059093010180930001892BC9F564E6BB
:100E400070E08FE30E94FD05909301018093000103
:100E5000892B71F584E690E00E94520664E670E00A
:100E600080E40E94A6059093010180930001892BE4
:100E7000F9F464E670E08CE00E94FD0590930101B6
:100E800080930001892BA1F464E670E080E00E9469
:100E9000FD059093010180930001892B49F464E6DC
:100EA00070E08FE30E94FD059093010180930001A3
:100EB00084E690E00E94520680910001089561113D
:100EC00008C0FC018281882321F08CEA91E00E9415
:100ED000150880E090E008958E3D2CE5920721F002
:100EE0008F3D9C4541F010C0FB018281882369F051
:100EF0000E94E22207C0FB018281882331F081E059
:100F00000E94231180E0089581E00895CF92DF923E
:100F1000EF92FF926B017C010E941A2256985E9814
:100F200025982D9826982E9827982F9890E0FC01C8
:100F30003197E730F105A8F4E35AFF4F0C9478336A
:100F4000259A2D9A0EC0259A2D9A269A2E9A09C076
:100F5000259A2D9A04C0259A2D9A269A2E9A279A78
:100F60002F9AC701B601FF90EF90DF90CF900895C0
:100F700081E008950C946C07CF93282F30E0F9019D
:100F8000EE51FC4FC491F901EE59FB4F24912223FD
:100F900059F081EE0E944E178C2F0E944E178C2F15
:100FA0000E94671881EE04C08C2F0E944E178C2F70
:100FB000CF910C9467180F931F93CF93DF93EC019D
:100FC000062FFE018491882359F19E012F5F3F4F28
:100FD000813041F4E901F9011491812F0E944E17EB
:100FE000812F0DC0823031F4E901F90184910E9412
:100FF0004E170AC0833031F4E901F90184910E944F
:10100000671802C00E94BC072196802F8823C9F26E
:10101000EFE9FFE03197F1F700C000008150F6CF13
:10102000DF91CF911F910F91089560E00C94DB0741
:101030000E946A22811106C00E947522811102C09D
:101040000E94E2220C94CE060C94B704282F2F7035
:1010500041F0822F90E02A3010F44D9608950697C3
:10106000089587E290E0089508950C9434080C9454
:10107000350808950E94DA1B0E9439082FEF84E397
:101080009CE0215080409040E1F700C000000C94AB
:101090003F24FF920F931F93CF93DF938C01FC01AA
:1010A000C081D18180919602811113C082818823F1
:1010B00049F0CE010E940D21F82E682FCE010E942A
:1010C000B02004C0CE010E94E020F82EBE018F2D7A
:1010D00004C0CE010E940D21BE010E94FC0AEC0159
:1010E000B8010E94BA07882309F47EC2B801CE0174
:1010F0000E94650D882309F477C2CB3CFCE5DF072D
:1011000041F4F8018281882309F46EC20E941A0F0B
:101110006BC2CC3C8CE5D80708F013C1C33C9CE5FE
:10112000D90761F4F8018281882309F45DC20E9425
:10113000DE218272F1F00E94301156C2C43CECE50F
:10114000DE07D0F0F8018281C73CFCE5DF0709F437
:10115000CDC008F0DDC0C53CECE5DE0709F4CCC02D
:1011600008F0D0C0882309F43FC20E94DE218272B9
:1011700011F30E94261138C2C531FCE5DF0708F0E3
:101180007EC0C2308CE5D80708F452C0F8018281D5
:10119000882309F459C00E946A22811102C00E946A
:1011A000E2220E94872290E09093AF038093AE03E7
:1011B000FE01E350FC45E231F10530F4EC59FF4FFC
:1011C0008091AE030C9478338091AE03816027C088
:1011D000826025C0846023C0806121C080621FC0FE
:1011E00080641DC080681BC08460886018C08E7FCA
:1011F00016C08D7F14C08B7F12C08F7E10C08F7D74
:101200000EC08F7B0CC08F770AC08B7F877F07C093
:1012100087FB222720F991E0922790FB87F98093A2
:10122000AE038091AE030E948B220E94DA1BDCC1C8
:10123000C1159CE5D90781F0C130DC45A9F081E0FA
:101240008093510280935202C801DF91CF911F9188
:101250000F91FF900C94B807F8018281882309F45C
:10126000C3C10E943A08C0C1F8018281882309F4F1
:10127000BBC180913503816080933503B5C1C63110
:10128000FCE5DF0739F50E94DE21282FF801828175
:1012900040910F0150911001882379F02A7A91E052
:1012A00009F490E090934C02911102C069E201C0F0
:1012B00065E3CA010E9440230AC080914C0281115B
:1012C00002C069E201C065E3CA010E944B230E948B
:1012D000AB218AC1C23CDC4509F0B1CFF801828163
:1012E000882309F481C10E94BF117EC1882309F4BB
:1012F0007BC10E94801078C1882309F475C10E94C7
:10130000491072C1882309F46FC10E9461106CC139
:10131000C93C9CE5D90731F4882309F465C10E94D2
:10132000A41062C1CA3CDC4530F4882309F45CC1D6
:101330000E94921059C1882309F456C10E94BF101F
:1013400053C1C33DFCE5DF0749F4F80182818823DE
:1013500009F44AC188E10E94231146C1C43D8CE5CD
:10136000D80708F087C0F8018281CF3CFCE5DF0791
:10137000A1F4882309F438C10E940C0F663071056E
:101380008105910540F00E940C0F683071058105C0
:10139000910508F4EECE86E0DECFC03D9CE5D9078E
:1013A00030F5CD3CECE5DE0729F4882309F41CC1B7
:1013B00081E0D1CFCE3CDC4530F4882309F414C160
:1013C0000E942F0F11C1882309F40EC10E940C0F37
:1013D000623071058105910540F00E940C0F653067
:1013E00071058105910508F4C4CE82E0B4CFC13DFA
:1013F0009CE5D907A1F4882309F4F6C00E940C0FDC
:101400006F3071058105910540F00E940C0F643129
:1014100071058105910508F4ACCE8FE09CCFC23DEB
:10142000DC45A0F4882309F4DFC00E940C0F69306A
:1014300071058105910540F00E940C0F6E30710519
:101440008105910508F495CE89E085CF882309F4BC
:10145000CBC00E940C0F653171058105910540F0EC
:101460000E940C0F673171058105910508F481CE4A
:1014700085E171CFC73DFCE5DF0781F5F801828189
:10148000882361F0109252020E94E323909350024D
:1014900080934F0280E20E94CF18A6C00E94DE21F6
:1014A00081FF05C081E080935102809352028091B8
:1014B000520281110FC080914F02909150020E9400
:1014C000EF23883C910530F487E20E944E1787E2B3
:1014D0000E94671880E20E94D61886C0C83D8CE53D
:1014E000D80708F04CC0F8018281C53DFCE5DF0754
:1014F00029F4882309F478C083E22DCFC63DDC456A
:10150000A0F4882309F470C00E940C0F69317105A2
:101510008105910540F00E940C0F62327105810532
:10152000910508F426CE89E116CF882351F0109258
:1015300051020E94E32390934E0280934D0282E079
:10154000AACF0E94DE2185FF05C081E08093510271
:10155000809352028091510281110FC080914D02FF
:1015600090914E020E94EF23883C910530F486E270
:101570000E944E1786E20E94671882E0ACCFCB3DF6
:10158000ECE5DE0731F4F8018281882369F180E01F
:1015900009C0CC3DFCE5DF0741F4F80182818823D6
:1015A00019F182E00E943E2B1FC0C83DDC4509F0C6
:1015B00046CEF8018281811165CF8091520281115E
:1015C00089CF80914F02909150020E94EF23883C76
:1015D000910508F07FCF80E20E94D61888E20E9431
:1015E0004E1788E20E94671880E0DF91CF911F912B
:1015F0000F91FF900895089596E0799FF0011124CE
:1016000094E5899FE00DF11D1124E60FF11DEE0F09
:10161000FF1FE651FE4F859194910895880F991F01
:10162000FC01EA51FE4F859194910895CF93DF9389
:101630000E94FC0A0E94C50CEC01811520E592076E
:10164000F0F5811530E4930708F021C1883E91053B
:1016500000F5803E910508F094C1883A910570F438
:10166000853A910508F0A3C08130910509F489C13C
:1016700008F440C1049708F084C13CC18D3B91053A
:1016800008F4A0C0803C910508F434C1805C910945
:10169000F0C08115904258F4C11581E0D80708F0D8
:1016A00070C1C03FD10508F425C1D0656AC1C1151C
:1016B00090E3D90708F0E1C0CE019F70DAC0811530
:1016C00025E5920708F043C0811534E5930708F03B
:1016D000F5C0811542E5940708F5C11581E5D807E5
:1016E00008F0D8C02C2F237081E090E002C0880F52
:1016F000991F2A95E2F79C689E0174E0369527951C
:101700007A95E1F72370922BCF70C695C69540E28B
:10171000C49FE0011124C82BD92B33C1869586952F
:101720009E0123703327C115D34508F0B8C040E2AD
:10173000849FC0011124C1E0D0E002C0CC0FDD1FA6
:101740002A95E2F78C2B9D2BEC01DC681AC18115E0
:101750002AE5920798F4811539E5930708F0B9C096
:101760008115964508F4AFC0C11588E5D80708F47F
:10177000C1C0DC2FCC27C06FD06A03C1C1159BE567
:10178000D90708F4B7C0C1152CE5D20708F4AFC0DB
:10179000CE0190568115904208F0ACC08D2F8F710C
:1017A0000E94420DDD27D0628F71D82BEAC0853AA6
:1017B000910509F4A2C0863A910509F0A1C0C2E8DA
:1017C000D0E4DFC0883A910509F49DC0893A9105BB
:1017D00009F49CC08A3A910509F49BC08B3A9105A3
:1017E00009F49AC08C3A910509F499C08B3B910594
:1017F00009F498C08C3B910509F497C08D3A910586
:1018000009F496C0803B910509F495C08E3A910584
:1018100009F494C08F3A910509F493C0813B910576
:1018200009F492C0823B910509F491C0833B910574
:1018300009F490C0843B910509F48FC0853B910564
:1018400009F48EC0863B910509F48DC0873B910554
:1018500009F48CC0883B910509F48BC0893B910544
:1018600009F48AC08A3B910509F489C0C0E0D4E438
:1018700088C00E940E0BEC0184C0CE019927D3FFD3
:1018800003C0EC01D86C7DC0EC01D06C7AC0DF7075
:10189000D06A77C0DC2FCC27C16FD06A72C040E21B
:1018A000849FC0011124C1E0D0E002C0CC0FDD1F35
:1018B0002A95E2F7C82BD92BDA6863C0D82FCC273A
:1018C000C46FD06A5EC0CF71DD27DC2FCC27D06219
:1018D00058C08F70806E90E0906A24E0D695C795CE
:1018E0002A95E1F7CF709C013C2BE9014AC0DD2726
:1018F000D06647C0C0E0D0E044C0C1E8D0E441C0F9
:10190000C3E8D0E43EC0C2EED4E43BC0C9EED4E4A8
:1019100038C0CAEED4E435C0C5EBD4E432C0C6EB5F
:10192000D4E42FC0C3EBD4E42CC0C4EBD4E429C06E
:10193000C7EBD4E426C0CCECD4E423C0CDECD4E493
:1019400020C0C3E8D5E41DC0CAE8D5E41AC0C2E986
:10195000D5E417C0C4E9D5E414C0C1E2D6E411C08F
:10196000C3E2D6E40EC0C4E2D6E40BC0C5E2D6E4BE
:1019700008C0C6E2D6E405C0C7E2D6E402C0CAE2A7
:10198000D6E4CE01DF91CF9108958238910549F1D7
:10199000B0F48133910509F458C048F489329105B7
:1019A00009F44EC08A32910509F454C00895853374
:1019B000910509F440C08933910599F00895833E5B
:1019C000910529F138F4803E910591F0823E910510
:1019D000A1F00895863E9105F9F0873E910531F119
:1019E00008952091AE0320FD3AC021FD38C008952E
:1019F0008091AE0380FD35C032C08091AE0382FF7E
:101A000032C08091AE0384FD30C083EE39C0809136
:101A1000AE0382FD28C0F5CF8091AE0383FF27C0BF
:101A20008091AE0384FD21C087EE2AC08091AE0371
:101A300083FD1DC0F5CF8091AE0385FD1AC01BC08C
:101A40008091AE0385FD17C014C08091AE0386FD62
:101A500014C015C08091AE0386FD11C00EC080EE8B
:101A60000FC089E30DC082EE0BC080E009C086EE96
:101A700007C089E205C085E303C08AE201C081E3B3
:101A800090E008959091AE0392FF0DC0282F287129
:101A9000283019F4877F846006C0282F24712430F1
:101AA00011F48B7F886093FF0DC0282F2871283197
:101AB00019F4877E846106C0282F2471243111F423
:101AC0008B7E886194FD877E0895CF93DF9381306C
:101AD00020E89207D0F0FB0122812223B1F0EC0133
:101AE00080915302811109C08CE090E00E948B33F9
:101AF0000E94890D81E0809353020E94900DCE01D7
:101B00009F770E94580E0E940C0E81E0DF91CF91CA
:101B1000089580935402682F8CE090E00C949F33DA
:101B2000E0910F01F091100180818093660381FFA5
:101B300003C081EE0E9467188091660385FF03C091
:101B400085EE0E9467188091660380FF03C080EED7
:101B50000E9467188091660384FF03C084EE0E9490
:101B600067188091660382FF03C082EE0E946718A7
:101B70008091660386FF03C086EE0E9467188091FD
:101B8000660383FF03C083EE0E946718809166039B
:101B900087FF03C087EE0E9467188091540282304D
:101BA00001F1A8F48823C9F0813079F580EE0E9414
:101BB0004E1781EE0E944E1788E10E944E1788E171
:101BC0000E94671881EE0E94671880EE1CC0843066
:101BD00081F08530D1F486EE01C082EE0E944E176E
:101BE00014C082EE0E944E1787E50E944E1787E5CB
:101BF0000AC086EE0E944E1786EE0E94671888E1A2
:101C00000E944E1788E10E9467188FE39CE90197B4
:101C1000F1F700C00000089580915402813049F02E
:101C200030F0823021F0853051F486EE06C082EE2D
:101C300004C08CE20E944E178CE20E9467188091CB
:101C4000660381FF03C081EE0E944E1780916603F8
:101C500085FF03C085EE0E944E178091660380FFCA
:101C600003C080EE0E944E178091660384FF03C07C
:101C700084EE0E944E178091660382FF03C082EEBD
:101C80000E944E178091660386FF03C086EE0E9475
:101C90004E178091660383FF03C083EE0E944E17A8
:101CA0008091660387FF03C087EE0C944E1708955A
:101CB000EF92FF921F93CF93DF937C01CCE0D0E0B3
:101CC00097010C2E02C0369527950A94E2F7122F41
:101CD0001F70812F0E9426080E944E17812F0E949C
:101CE00026080E9467182497CC3F8FEFD80741F74A
:101CF000DF91CF911F91FF90EF900895EF92FF92A7
:101D00000F931F93CF93DF93E901662309F44BC030
:101D1000242F30E0EFEFF0E0E61BF109B901E69F78
:101D20009001E79F300DF69F300D1124232F8B017A
:101D3000031B11095CE3E52EF12CB7010E9450331F
:101D4000FB01BC01069FC001079F900D169F900DDF
:101D50001124B7010E945033E230F105B1F040F494
:101D6000309779F0319711F5832F242F461B21C02E
:101D7000E430F105A1F068F03597C1F4842F861B9B
:101D800018C0832F262F230F14C0862F830FE42F14
:101D900003C0E42FE61B842F432F2E2F0AC0842F6D
:101DA000462F430F06C0842F242F03C080E020E07D
:101DB00040E0E42FF0E0E250FB4F4491E22FF0E0EE
:101DC000E250FB4F9491E82FF0E0E250FB4FE4919A
:101DD00049839883EA83DF91CF911F910F91FF9000
:101DE000EF90089588E090E00C949333AB01BC0130
:101DF00088E090E00C94B133E7E6F3E083E0808381
:101E0000109268038FEF82838383148260817181D3
:101E1000828193810C94F60E6091670360FF06C087
:101E200066956F7370E080E090E0089560E070E088
:101E3000CB01089580916B0390E001968430910569
:101E400014F083E090E080936B03609167037091DE
:101E500068038091690390916A030C94F60E809157
:101E60006B0390E0019797FF02C080E090E0843020
:101E7000910514F083E090E080936B036091670319
:101E8000709168038091690390916A030C94F60E37
:101E90008091670380FF06C06FE070E08CE693E0FE
:101EA0000C94731580E090E0FC01E459FC4F118222
:101EB0001082128204968C339105B1F7EDCF909188
:101EC000670390FF0FC020E030E0F901E459FC4FB8
:101ED0008183608342832C5F3F4F2C333105A9F708
:101EE0000C94480F0895CF93DF9300D000D0CDB766
:101EF000DEB72091670320FF0AC09E012F5F3F4F8E
:101F00000E947E0E4B8169818A810E945F0F0F9033
:101F10000F900F900F90DF91CF9108955F926F9285
:101F20007F928F929F92AF92BF92CF92DF92EF9269
:101F3000FF920F931F93CF93DF9300D000D0CDB7C4
:101F4000DEB78C01E62EF42E522E8091670380FFBF
:101F500089C0982F9E77923061F49E012F5F3F4F8A
:101F6000C8010E947E0E4B8169818A810E945F0FA9
:101F700059C0E82FE695EF739EE39E0F9F73943050
:101F800018F4F0906A034EC09AE39E0F9F73993045
:101F900068F4881F8827881F90916803292F220FD3
:101FA000022F082B97FB112710F93CC087E28E0FF8
:101FB0008F738A30B8F5F0E07997E0FD02C021E038
:101FC00001C02FEFEE7FEC50FB4F859194916FE0B5
:101FD00070E00E94503326034001279F900C11248B
:101FE000580188E9A81A8EEFB80A8CE6C82E83E05B
:101FF000D82E98E6692E77247394C501B3010E9408
:10200000503396014F2D6E2D0E947E0EA80CB91CE8
:1020100084E0C80ED11C88EAC81683E0D80669F7A8
:102020000E94480F8091670300FB87F98093670344
:10203000902F9695809168038078892B10FB87F903
:1020400080936803E0926903F0926A03552051F08F
:1020500060916703709168038091690390916A03AE
:102060000E94F60E0F900F900F900F90DF91CF917E
:102070001F910F91FF90EF90DF90CF90BF90AF90A6
:102080009F908F907F906F905F90089521E00C94C7
:102090008E0FE7E6F3E02081221F2227221F3091D6
:1020A0006803432F440F842F822B37FB992790F925
:1020B0000C9668E671E00E946433438162810C945F
:1020C000461020916703221F2227221F30916803A8
:1020D000432F440F842F822B37FB992790F98C30A4
:1020E00091051CF4845A9E4F01C00C9768E671E07C
:1020F0000E94643340916A03609169030C94461016
:10210000E7E6F3E08081881F8827881F90916803A5
:10211000292F220F97FB992790F943816FEF822B8C
:102120000C944610E7E6F3E08081881F8827881F1B
:1021300090916803292F220F97FB992790F94381EB
:1021400060E0822B0C94461040916A03842F90E04B
:10215000843F910514F4445F01C04FEF8091670301
:10216000881F8827881F90916803292F220F97FBCB
:10217000992790F960916903822B0C944610409145
:102180006A03842F90E00C9714F04C5001C040E09B
:1021900080916703881F8827881F90916803292FE3
:1021A000220F97FB992790F960916903822B0C9479
:1021B000461020E00C948E0FCF939091670390FF10
:1021C00040C09178811102C0926007C0853210F042
:1021D000986403C08F73880F982B909367036623CE
:1021E00051F0609167037091680380916903909149
:1021F0006A030E94F60EC09167036C2F66956F7399
:1022000070E04BE050E084E091E00E947E33892B47
:1022100019F01092720203C081E080937202CC1F09
:10222000CC27CC1F90916803892F880F97FB9927A3
:1022300090F940916A03609169038C2BCF910C94C3
:10224000D910CF91089561E00C94DC108091670360
:1022500086958F738F5F853208F081E00C9423118F
:102260008091670386958F73815009F484E20C9402
:102270002311E7E6F3E080818160808386958F7388
:102280000C94231160E00C94DC1080913503816084
:10229000809335030E946A22811104C00E94E222C9
:1022A0000E94FC0E0E94F20E609367037093680315
:1022B0008093690390936A036E7761F40E94FC0E29
:1022C0000E94F20E60936703709368038093690322
:1022D00090936A0381E0809372028091670380FF8C
:1022E00004C086958F730C944211089590916703F2
:1022F00090FF0DC02F3058F494E0299FF001112475
:10230000E459FC4F8183608342830C94480F089505
:102310001F93CF93DF9300D000D0CDB7DEB73091BD
:10232000670330FF0CC0122F9E012F5F3F4F0E94AA
:102330007E0E212F4B8169818A810E9476110F9038
:102340000F900F900F90DF91CF911F910895E7E6C6
:10235000F3E080818E7F80836081718182819381AF
:102360000E94F60E109272022FEF80E792E0215049
:1023700080409040E1F700C000000C94480F80912D
:10238000670380FD0C94A7110C943911CF93C82FCB
:1023900080917002909171020E94EF23EC2FF0E087
:1023A000E051FB4FE491F0E08E179F0708F443C023
:1023B0000E94E323909371028093700260916F02F8
:1023C00070E080E090E00E94513120E030E04FE783
:1023D00053E40E9474302BED3FE049E450E40E9446
:1023E0007A320E94E7320E94EE302BE43AE34EE26A
:1023F0005FE30E94073020EF3BEF48ED52E40E947C
:102400007A320E942031462F80916703881F8827E7
:10241000881F90916803292F220F97FB992790F925
:1024200060916903822B0E94730F80916F0290E08C
:10243000019680936F02CF910895CF93C82F80911A
:102440006D0290916E020E94EF23EC2FF0E0E351B9
:10245000FB4FE491F0E08E179F07E8F00E94E32322
:1024600090936E0280936D0240916A0360916903BC
:1024700080916B0290916C020E94730F80916B02AD
:1024800090916C02019668E671E00E94503390933F
:102490006C0280936B02CF910895CF92DF92FF92EE
:1024A0000F931F93CF93DF93F82E80916902909141
:1024B0006A020E94EF23EF2DE695F0E0E651FB4F14
:1024C000E491F0E08E179F07E8F10E94E3239093D8
:1024D0006A02809369020CE613E0C0E0D0E088E66F
:1024E000C82EDD24D39480916702909168028C0FEE
:1024F0009D1FB6010E945033980140916A0360917C
:1025000069030E947E0E68960C5F1F4FC83681E0FB
:10251000D80749F70E94480F20916702309168025E
:10252000F0FE0AC0C9010196BE010E94503390938B
:1025300068028093670206C0215031093093680217
:1025400020936702DF91CF911F910F91FF90DF9051
:10255000CF900895AF92BF92CF92DF92EF92FF9209
:102560000F931F93CF93DF93C82F80FF02C01FEFFD
:1025700001C011E080916502909166020E94EF23F4
:10258000C695EC2FF0E0E951FB4FE491F0E08E1797
:102590009F0708F466C00E94E3239093660280932D
:1025A00065022CE6C22E23E0D22E3EE6E32E33E077
:1025B000F32EC0E0D0E0F70131971082F6011082CF
:1025C000F701108294E0A92EB12C00E08091640202
:1025D000800F87FD815F082E000C990BC817D90763
:1025E000E9F480916A038A9DA0018B9D500D11240E
:1025F000559547955595479580916703881F88277E
:10260000881F90916803592F550F97FB992790F9D0
:10261000960160916903852B0E947E0E010FF1E007
:10262000AF1AB10899F6219684E0C80ED11CE4E0F7
:10263000EE0EF11CCF30D10509F0BDCF0E94480F3E
:1026400080916402113031F4811102C08EE007C024
:10265000815005C090E00196BE010E9464338093D2
:102660006402DF91CF911F910F91FF90EF90DF9067
:10267000CF90BF90AF9008950F931F93CF93DF93A8
:10268000C82F80916202909163020E94EF23EC2F89
:10269000F0E0EC51FB4FE491F0E08E179F0708F457
:1026A00064C00E94E323909363028093620280E0FF
:1026B00090E0FC01E459FC4F1182108212820496D2
:1026C0008C339105B1F7C0E0D0E00FE010E0CE010F
:1026D000B8010E946433FC0180916102082E000C55
:1026E000990BEE0FFF1FEE0FFF1FC817D907FCF065
:1026F00080910301082E000C990B8C179D07BCF0EC
:102700009F0124593C4F80916703881F8827881FA9
:1027100090916803592F550F97FB992790F9409195
:102720006A0360916903852B0E947E0E05C0E459FF
:10273000FC4F1182108212822196CF30D10539F6DA
:102740000E94480F8091020190916102980F90932E
:10275000610220910301280F20930301121614F443
:102760009E301CF0819580930201DF91CF911F91E3
:102770000F910895EF92FF920F931F93CF93DF93E2
:1027800080915F02909160020E94EF23883E934007
:10279000D0F10E94E3239093600280935F02C09186
:1027A0005D02D0915E022196C170DD27D0935E025A
:1027B000C0935D028CE6E82E83E0F82E10E008E777
:1027C000812F8695FE01E80FF11DCF0181709927B9
:1027D000970140916A0360916903FC010E9FC0015B
:1027E0000F9F900D11240E947E0E1F5FF4E0EF0EEC
:1027F000F11C1F3029F7DF91CF911F910F91FF90AE
:10280000EF900C94480FDF91CF911F910F91FF90A3
:10281000EF900895CF93DF9300D000D0CDB7DEB70F
:1028200080915B0290915C020E94EF23E2EEF4E063
:102830002591349182179307C0F180915A0281113A
:102840000CC09E012F5F3F4F4FEF6FEF80E090E095
:102850000E947E0E8A8180935A020E94E323909305
:102860005C0280935B0280915902813051F028F024
:10287000823061F440915A020AC080915A0240E0CD
:1028800007C060915A0240E080E003C040E080E071
:1028900060E00E945F0F8091590290E0019663E032
:1028A00070E00E946433809359020F900F900F9054
:1028B0000F90DF91CF910895CF93DF9380915702CE
:1028C000909158020E94EF23843F914008F444C045
:1028D0000E94E3239093580280935702C0E0D0E017
:1028E00020915502309156028091670390916803C0
:1028F000C730D1051CF4232B79F002C0232B61F4DF
:10290000881F8827881F392F330F97FB992790F945
:102910002C2F40916A030AC0881F8827881F392FEF
:10292000330F97FB992790F92C2F40E060916903B2
:10293000832B0E9488112196CF30D10589F60E9401
:10294000480F809155029091560201968170992707
:102950009093560280935502DF91CF910895809114
:1029600072028823D9F190916703892F86958F731E
:102970002EE3280F2F73243018F482500C94C611C4
:102980002AE3280F2F73233018F486500C941D125D
:1029900027E3280F2F73263018F489500C944D121A
:1029A00021E3280F2F73263018F48F500C94AA12AD
:1029B0002BE2280F2F73233018F485510C943C130D
:1029C000892F8E77803311F40C94BA13863411F466
:1029D0000C940A14883411F40C945C140895882320
:1029E00019F05198599A02C0519A59985098589A8A
:1029F00095E09A95F1F70000509A589895E09A95CD
:102A0000F1F70000882311F0519A599885E08A95D2
:102A1000F1F7000008958BB18C7F8BB95098589ACC
:102A20005198599A85E08A95F1F7000008958AB186
:102A30008C7F8AB985E08A95F1F70000519A599800
:102A400085E08A95F1F70000509A589885E08A95BC
:102A5000F1F7000008955098589A85E08A95F1F7AB
:102A600000005198599A85E08A95F1F70000089581
:102A7000CF93DF93D82FC8E08D2F80780E94EF147A
:102A8000DD0FC150C9F780E00E94EF1485E08A9500
:102A9000F1F7000085E08A95F1F7000080E0DF9112
:102AA000CF9108952BB1342F309523233BB1432B85
:102AB0003FB7F894FC01680F791FE617F70789F014
:102AC000819198E04BB9000000C087FF2BB9880FB7
:102AD000000000C000C000C02BB900C09A9591F75B
:102AE000ECCF3FBF0895AF92BF92CF92DF92EF92AB
:102AF000FF920F931F93CF93DF938C01EB01CFB61F
:102B0000D090BC00F8948091BC008B7F8093BC0077
:102B10000E940B150E94171584E80E943815CC0FEF
:102B2000DD1FCC0FDD1F78015801AC0EBD1EEA146D
:102B3000FB0431F0F70181917F010E943815F7CF36
:102B40000E942B15CFBED092BC00579A40E8BE0120
:102B5000C801DF91CF911F910F91FF90EF90DF900F
:102B6000CF90BF90AF900C945215909378028093C1
:102B700077020895E0917702F0917802309721F082
:102B80000190F081E02D099480E00895E0917702B2
:102B9000F0917802309721F00280F381E02D0994C2
:102BA0000895E0917702F0917802309721F0048047
:102BB000F581E02D099408952091750230917602F7
:102BC0008217930771F09093760280937502E091DB
:102BD0007702F0917802309721F00680F781E02D9E
:102BE000099408952091730230917402821793071B
:102BF00071F09093740280937302E0917702F091E8
:102C00007802309721F00084F185E02D0994089531
:102C100008950C94081681E008950E94DA2385B780
:102C2000806885BF85B7806885BF0E94B9040E940F
:102C300071240C944511CF92DF92EF92FF920F9383
:102C40001F93CF93DF93CDB7DEB72B970FB6F894D2
:102C5000DEBF0FBECDBF0E942B050E940B16811157
:102C600011C08FEF89838A831B820E94E3238160D6
:102C7000782F9D838C8349815A816B818D810E943D
:102C8000FF1656C08AE7C82E82E0D82E00E010E07A
:102C9000E02E802F0E949905F60141916F01F42EDC
:102CA000F82631F40F5F1F4F0E30110589F7D9CF89
:102CB0009091350391FF04C08B870E949F058B85FF
:102CC00020E030E04F2D50E0922FBA01022E02C0DA
:102CD000759567950A94E2F760FF24C02E83EF8212
:102CE00021E030E0690102C0CC0CDD1C9A95E2F7CE
:102CF00090E08C219D21892B09F420E028870E94F7
:102D0000E3238160782F9A8789874E815F81688568
:102D10008A850E94FF16F801E658FD4F8081C8267B
:102D2000C08206C02F5F3F4F2630310569F6BACF0B
:102D30000E940426109179020E94BA151817A1F07A
:102D40000E94BA15809379022B960FB6F894DEBFD5
:102D50000FBECDBFDF91CF911F910F91FF90EF90EC
:102D6000DF90CF900C9437082B960FB6F894DEBF07
:102D70000FBECDBFDF91CF911F910F91FF90EF90CC
:102D8000DF90CF900895DC0111962C9111978C91D2
:102D9000682F70E041E050E001C0440F8A95EAF7E7
:102DA00012968C91129730E0882329F08091980236
:102DB0008823E9F006C0F901E857FD4F908194237C
:102DC000B1F086E0829FF001839FF00D1124E60FA1
:102DD000F71FEE0FFF1FEF5DFE4F808191818D93F6
:102DE0009C93F901E857FD4F8081482B06C0F901FB
:102DF000E857FD4F40958081482340830895CF9345
:102E0000DF93CDB7DEB72B970FB6F894DEBF0FBEBA
:102E1000CDBF942F4F83252F588769877A878B875B
:102E20004A855B85452B21F02F3F09F59F3FF9F43B
:102E3000DE01119686E0FD0111928A95E9F785E0A1
:102E4000FE01379601900D928A95E1F749815A81EA
:102E50006B817C818D819E810E94811E2B960FB695
:102E6000F894DEBF0FBECDBFDF91CF910895CE01A4
:102E700007960E94C316DCCFFC01808191810E94DD
:102E80004C2192959F70963041F48091980291E088
:102E9000892780939802909397020895CF93DF93A8
:102EA0001F92CDB7DEB7882309F40DC1682F823891
:102EB000C1F40E94BA1581FD06C169E380910F013A
:102EC000909110010E9440230E94AB212FEF81EED0
:102ED00094E0215080409040E1F700C0000069E399
:102EE00019C0833811F50E94BA1580FDECC063E566
:102EF00080910F01909110010E9440230E94AB210C
:102F00002FEF81EE94E0215080409040E1F700C027
:102F1000000063E580910F01909110010E944B2306
:102F20000F90DF91CF910C94AB218438C1F40E94B3
:102F3000BA1582FDC8C067E480910F01909110011D
:102F40000E9440230E94AB212FEF81EE94E021509C
:102F500080409040E1F700C0000067E4DBCF8CEFD9
:102F6000860F813A70F4862F69830E943A2869811E
:102F70008111A9C080910F01909110010E944023FE
:102F8000CFCF80E2860F883048F4677081E001C0BF
:102F9000880F6A95EAF70E94E121C2CF8BE5860F80
:102FA000833088F4653A29F0663A31F083E890E09E
:102FB00005C081E890E002C082E890E00F90DF91C8
:102FC000CF910C94DC1588E5860F853108F071C02F
:102FD000683A61F1693A69F16A3A71F16B3A79F1EB
:102FE0006C3A81F16B3B89F16C3B91F16D3A99F14F
:102FF000603BA1F16E3AA9F16F3AB1F1613BB9F1D1
:10300000623BC1F1633BC9F1643BD1F1653BD9F14E
:10301000663BE1F1673BE9F1683BF1F1693BF9F1AE
:103020006A3B09F43FC080E090E03EC082EE90E051
:103030003BC089EE90E038C08AEE90E035C085EB69
:1030400090E032C086EB90E02FC083EB90E02CC084
:1030500084EB90E029C087EB90E026C08CEC90E0F8
:1030600023C08DEC90E020C083E891E01DC08AE889
:1030700091E01AC082E991E017C084E991E014C0A0
:1030800081E292E011C083E292E00EC084E292E01D
:103090000BC085E292E008C086E292E005C087E2BC
:1030A00092E002C08AE292E00F90DF91CF910C94FF
:1030B000F215603F40F0862F0E940C250F90DF91A3
:1030C000CF910C94F9250F90DF91CF91089588232B
:1030D00009F464C0823879F40E94BA1581FF5EC099
:1030E00069E380910F01909110010E9440230E949A
:1030F000AB2169E310C08338B1F40E94BA1580FF98
:103100004DC063E580910F01909110010E94402312
:103110000E94AB2163E580910F01909110010E9404
:103120004B230C94AB21843879F40E94BA1582FFAA
:1031300035C067E480910F01909110010E944023F7
:103140000E94AB2167E4E7CF9CEF980F913A10F40F
:10315000682FE1CF90E2980F983050F4877091E09B
:1031600001C0990F8A95EAF7892F0E94E721D9CFEC
:103170009BE5980F933020F480E090E00C94DC15F0
:1031800098E5980F953120F480E090E00C94F215CA
:10319000803F20F00E9474250C94F925089588231F
:1031A00021F00E94E1210C94AB210895882321F0A5
:1031B0000E94E7210C94AB2108958F929F92AF92C9
:1031C000BF92DF92EF92FF920F931F93CF93DF9303
:1031D0007C01D62FC72FFC01058102950F7012814B
:1031E00011110E94FE210E94A421882379F011234D
:1031F00069F080E28D0F883048F082E00E948D21D6
:103200000E94A42191E0D82ED92601C0D12CAC2E49
:10321000A2948FE0A822B12CF501EA58FF4F0C943C
:1032200078338C2F807FCF70882311F0C295C07FB8
:10323000112399F0CC2309F4C8C180E28D0F8830A6
:1032400010F0D11104C08C2F0E94E12103C08C2FFB
:103250000E94F1210E94AB21B8C18D2F0E946718F6
:10326000CC2309F42EC280E28D0F883010F0D111EA
:1032700004C08C2F0E94E72103C08C2F0E94F721ED
:103280000E94AB211EC28C2F807FCF70803211F044
:10329000C295C07FDD2319F0D130C9F021C01123C0
:1032A00071F0002341F0013031F40E9417228C2B81
:1032B0000E94112206C20E9417228C2B3FC10023BC
:1032C00019F0013009F4FDC10E94142211C011232C
:1032D00021F0023008F0F5C107C00111F2C108C0A9
:1032E000112321F0011171C18C2F28C101117EC160
:1032F0008C2F2AC18C2F86958695837090E000973D
:1033000019F0019761F0DDC1112321F08D2F9C2F61
:10331000937002C080E090E00E94DC15E2C11123AE
:1033200021F08D2F9C2F937002C080E090E00E94CE
:10333000F215D7C11123F9F0D53F51F0D63F71F006
:10334000D43FA9F48091A8039091A90381600BC098
:103350008091A8039091A903826005C08091A80381
:103360009091A90384609093A9038093A8038D2F63
:103370000E940C251EC0D53F51F0D63F71F0D43FBE
:10338000A9F48091A8039091A9038E7F0BC080912E
:10339000A8039091A9038D7F05C08091A803909107
:1033A000A9038B7F9093A9038093A8038D2F0E947C
:1033B00074250E94F92595C18C2F837009F050C0A7
:1033C00011118BC18D2F829586958770880F880F7C
:1033D0009D2F9F70892E912CA12CB12C082E04C0FA
:1033E000880C991CAA1CBB1C0A94D2F7D4FF14C0E9
:1033F0000FE010E020E030E0B901A80104C0440F64
:10340000551F661F771F8A95D2F7CB01BA016095C9
:1034100070958095909503C060E070E0CB01C695F3
:10342000C695C370D0E0C230D10561F0C330D1057C
:1034300081F0682979298A299B29219771F00E94B6
:10344000C61F4BC1682979298A299B290E94D81F48
:1034500044C10E94C61FC501B4010E94B41F3DC1F2
:10346000112319F08C2F817001C08695882309F4EF
:1034700034C18D2F829586958770880F880F9D2F78
:103480009F70892E912CA12CB12C082E04C0880C81
:10349000991CAA1CBB1C0A94D2F7D4FF14C00FE0DD
:1034A00010E020E030E0B901A80104C0440F551F2E
:1034B000661F771F8A95D2F7CB01BA016095709588
:1034C0008095909503C060E070E0CB01C695C695ED
:1034D000C3704C2F50E04230510569F04330510524
:1034E00089F0682979298A299B294130510571F091
:1034F0000E948B20F2C0682979298A299B290E9481
:103500009D20EBC00E948B20C501B4010E94792050
:10351000E4C08D2F90E0FC01E05EF109E531F1059A
:1035200008F04FC0EA57FF4F0C947833DF708C2FB0
:103530008F71112331F00E9412208D2F0E94CF181D
:10354000C0C00E9433208D2F0E94D618BAC011230C
:1035500039F00111B6C08C2F8F710E945820B1C074
:10356000023008F0AEC0F7CF112339F08C2F8F71E5
:103570000E941220A6C01123C9F38C2F8F710E94C4
:1035800033209FC0112329F08C2F8F710E94FD1FC3
:1035900098C00E94F81F95C0112349F0CF718C2F5D
:1035A0000E94122063E08C2F0E9484218AC081E057
:1035B0000E948D21023008F484C082E00E948D2197
:1035C00080C0112331F0002389F28D2F0E944E1705
:1035D00078C0002391F2D93349F45FEF67EE73E0CE
:1035E000515060407040E1F700C000008D2F0E94F4
:1035F000671867C04C2F4F706D2FC7010E945F077F
:103600000E94251F6EC0D23FB1F028F4D03F49F090
:10361000D13FF9F028C0D43FB9F058F0D53F71F050
:1036200022C0112309F447C09091980281E08927B4
:1036300008C081E01827109398023DC011113BC0CB
:1036400081E08093980237C0111135C01092980222
:1036500032C0112329F080919702882329F329C0D1
:10366000002311F328C0809197020023C1F0882322
:1036700041F09091980281E08927809398021092FE
:1036800097028D2F112319F00E944E1714C00E942B
:10369000671886E0F70111928A95E9F70CC0882334
:1036A00051F0111108C09091980281E08927809310
:1036B0009802109297024C2F4F706D2FC7010E94F5
:1036C000FB0AF8E0AF16B10441F05CF04AE0A41A3E
:1036D000B10852E0A516B10420F40E94BA150E9468
:1036E0003708DD20E1F00E94802180FD18C0F7013D
:1036F00012820E947A210E941220C7010E949B1B05
:103700000E947A21DF91CF911F910F91FF90EF904E
:10371000DF90BF90AF909F908F900C943320DF91FB
:10372000CF911F910F91FF90EF90DF90BF90AF90DE
:103730009F908F9008950F931F93CF93DF93EC0189
:10374000888199812B813C81232BB9F09F3F11F413
:103750008F3F99F0CE010E944908882371F068815B
:1037600079818A810E9457218C010E94AF200E949A
:10377000B11FB801CE010E94DD18DF91CF911F91DA
:103780000F9108950E94FE210E940E2280910F0148
:10379000909110010E9456230E94AB210E949F2607
:1037A0000E94F92580E090E00E94DC1580E090E026
:1037B0000C94F2150E94EE210C94C21B0E944C2125
:1037C000E92FE295EF70F0E03297EE30F105B0F4BA
:1037D000E556FF4F0C947833803F91F018F4803E0B
:1037E00068F40EC0843F51F40BC0803E48F0813F26
:1037F00029F406C093FB882780F9089580E0089596
:1038000081E00895CF93DF9300D000D01F92CDB711
:10381000DEB70F900F900F900F900F90DF91CF9128
:103820000895CF93DF9300D000D000D0CDB7DEB79E
:1038300026960FB6F894DEBF0FBECDBFDF91CF91B5
:1038400008951F93CF93DF93C091990216E0809162
:103850009A02C81799F0D0E01C9FF0011D9FF00D4F
:103860001124E556FD4F408151816281738184812D
:1038700095810E94111C2196C770E9CFDF91CF91ED
:103880001F9108954091CB025091CC026091CD02DE
:103890007091CE028091CF029091D0020C94111CB5
:1038A0008091D00282958F7009F054C08091CD0232
:1038B000882309F44FC080919902A0919A026091E7
:1038C000CB027091CC024091CE025091CF02B6E073
:1038D0008A1709F43FC090E041155105C1F17F3FBF
:1038E00011F46F3FA1F1B89FF001B99FF00D1124C1
:1038F000E556FD4F218172132AC02081621327C033
:103900002281211124C0238134812417350710F42A
:1039100021503109241B350B283C3105C0F420917E
:10392000D0022F7020612093D00226E0289FF00162
:10393000299FF00D1124E056FD4F80818F7080612A
:1039400080838BEC92E00E949B1B0C94211C0196BF
:103950008770BECF0895CF92DF92EF92FF920F93C0
:103960001F93CF93DF93CDB7DEB762970FB6F8946E
:10397000DEBF0FBECDBF8C0185E0F801DE011D96D4
:1039800001900D928A95E1F7D8014C9111965C91C6
:10399000119712966C9112971396CD90DC90149714
:1039A0003091CB027091CC028091CE029091CF02E7
:1039B000009709F46BC17F3F19F43F3F09F466C1DA
:1039C000E090CD02EE2009F4C0C02091D002C816CC
:1039D000D90628F0F601E81BF90BCF0104C0809549
:1039E00090958C0D9D1DFF24F394883C910578F0F3
:1039F000F12C207F09F0C6C07C2DD98AC88A89891C
:103A00000E94021C8BEC92E00E949B1BB1C0822F93
:103A1000807F09F046C0751314C0341312C06111C1
:103A200010C02F7020612093D0020E94421C8BECAA
:103A300092E00E949B1B8091D002D80115968C9336
:103A40002EC0CD2819F15F3F11F44F3FF9F0F62E4B
:103A500061111CC08091990220919A0236E0821770
:103A600009F45AC090E0389FF001399FF00D1124FD
:103A7000E556FD4F7181571306C07081471303C08F
:103A80007281711103C001968770E9CFF62E66230B
:103A900009F427C18091D00281608093D002F12C7B
:103AA00020C1751308C0341306C0611104C0809191
:103AB000D002D801C3C04D875E878D859E856A8BF5
:103AC0000E94DE1B6A898823E1F16623D1F12091EF
:103AD000D002822F82958F7090E0029774F08091CF
:103AE000CB029091CC0298878F831986DB86CA8699
:103AF0002C87CE0107960E949B1B86E0F801ABEC59
:103B0000B2E001900D928A95E1F70E94501C0E944C
:103B1000421CFF24F394E5C04D875E878D859E850A
:103B20000E944C21292F22952F7030E02230310540
:103B30000CF0CBC09F7009F0C5C0805E883008F4DF
:103B4000D0C0C8010E949B1BE4CFC816D90608F458
:103B500053C0F601E81BF90BCF01883C910508F42E
:103B600050C0F12C7C2DD98AC88A89890E94021CF8
:103B7000EBECF2E086E0DF011D928A95E9F70E9406
:103B8000421CAFC0751314C0341312C0611110C0B1
:103B90008091D002F8018583C8010E949B1B86E0BA
:103BA000EBECF2E0DF011D928A95E9F7FE2C99C05B
:103BB0004D875E878D859E856A8B0E94DE1B6A8994
:103BC000882309F4BECF662309F4BBCF2091D0022D
:103BD000822F82958F7090E002970CF48ECF8091A7
:103BE000CB029091CC029A8389831B82DD82CC82A6
:103BF0002E83CE0101967FCF809590958C0D9D1DD3
:103C0000ACCFF62E662309F49CCF75132EC0341367
:103C10002CC02091D00220FD1FC0822F82958F7072
:103C2000D9F0D80115962C9315978F3049F08F5FF6
:103C3000982F9295907F822F8F70892B15968C9359
:103C4000C8010E949B1B86E0F801ABECB2E001903A
:103C50000D928A95E1F793CF86E0F801ABECB2E0E4
:103C600001900D928A95E1F73CC04D875E878D8566
:103C70009E850E94DE1B811140CF8091D002816021
:103C80008093D002C8010E949B1B2BC0662309F4BD
:103C900058CF4D875E878D859E850E94DE1BF82E4E
:103CA000882309F44ECF86E0F801ABECB2E0019036
:103CB0000D928A95E1F78BEC92E00E943C170E94EE
:103CC000501C5DCF811139CF0CC0243031050CF070
:103CD00038CF9F7009F431CFF8019581907F09F0BA
:103CE0002CCF8F2D62960FB6F894DEBF0FBECDBFDE
:103CF000DF91CF911F910F91FF90EF90DF90CF90C8
:103D000008951F93CF93DF93CDB7DEB72C970FB6EF
:103D1000F894DEBF0FBECDBF4F83588769877A877F
:103D20008B879C87CE0107960E94AB1C882369F085
:103D30008F8198852A853B85232BF1F19F3F09F0E0
:103D400063C08F3F09F060C037C086E0FE01379640
:103D5000DE01119601900D928A95E1F76F817885C9
:103D6000EA85FB85309741F17F3F11F46F3F21F1E8
:103D700020919A0230E0C9010196877099274091FD
:103D8000990250E08417950709F447C069837A8344
:103D9000FD83EC8396E0929FD001939FB00D112498
:103DA000A556BD4FFE01319601900D929A95E1F70F
:103DB00080939A020E94211C16E0809199029091B2
:103DC0009A028917C1F1189FC001112485569D4F91
:103DD0000E94AB1C882379F1E09199021E9FF001AB
:103DE0001124E556FD4F40815181628173818481A8
:103DF00095810E94111C8091990290E00196877034
:103E0000992780939902D9CF4F81588569857A8502
:103E10008B859C850E94111CCFCF0E94DA1B1092CB
:103E20009A0210929902EBECF2E086E0DF011D921B
:103E30008A95E9F7C1CF2C960FB6F894DEBF0FBE76
:103E4000CDBFDF91CF911F910895EF92FF920F9315
:103E50001F93CF93DF938C01892B09F46CC0F12C55
:103E6000EE24E394E8012196F8018491843740F42C
:103E7000843008F051C0813081F0823019F15BC08C
:103E8000853709F444C0A8F19CE7980F903708F0F3
:103E900052C08F770E94671841C00E5F1F4FFE010E
:103EA000C49180E28C0F883048F4C7708E2D01C019
:103EB000880FCA95EAF70E94012214C08C2F0E9435
:103EC0004E172DC00E5F1F4FFE01C49180E28C0F74
:103ED000883058F4C7708E2D01C0880FCA95EAF754
:103EE0000E9407220E94AB211AC08C2F0E946718E3
:103EF00016C00E5F1F4FFE01C491CC2381F08FE9E5
:103F00009FE00197F1F700C00000C150F6CF0E5FAF
:103F10001F4FFE01F49003C00E944E178E018F2D9B
:103F2000882309F49FCFEFE9FFE03197F1F700C054
:103F300000008150F5CFDF91CF911F910F91FF903D
:103F4000EF90089508950C94A21F0E94A31F609300
:103F50000C0370930D0380930E0390930F030C9446
:103F6000C21B08950C94A51F0F931F9300910C037F
:103F700010910D0320910E0330910F03602B712BD4
:103F8000822B932B1F910F910C94A51F0F931F93BE
:103F900000910C0310910D0320910E0330910F033B
:103FA00060237123822393231F910F910C94A51FEB
:103FB0000F931F9300910C0310910D0320910E039A
:103FC00030910F0360277127822793271F910F914C
:103FD0000C94A51F0C9486070E94EA1F60930803A7
:103FE0007093090380930A0390930B030C94C21BF4
:103FF00060E070E0CB010C94EC1F0F931F9341E045
:1040000050E060E070E08A019B0104C0000F111FC6
:10401000221F331F8A95D2F7C901B8011F910F9152
:104020000C94EC1F0F931F9341E050E060E070E0B0
:1040300004C0440F551F661F771F8A95D2F78091E1
:10404000080390910903A0910A03B0910B038A0120
:104050009B01082B192B2A2B3B2BC901B8011F915F
:104060000F910C94EC1F0F931F9341E050E060E020
:1040700070E004C0440F551F661F771F8A95D2F762
:104080004095509560957095809108039091090333
:10409000A0910A03B0910B038A019B010823192305
:1040A0002A233B23C901B8011F910F910C94EC1FE7
:1040B0000F931F9341E050E060E070E004C0440FB4
:1040C000551F661F771F8A95D2F78091080390913C
:1040D0000903A0910A03B0910B038A019B010827F1
:1040E00019272A273B27C901B8011F910F910C946A
:1040F000EC1F0F931F930091080310910903209167
:104100000A0330910B03602B712B822B932B1F9191
:104110000F910C94EC1F0F931F93009108031091C3
:10412000090320910A0330910B036023712382233A
:1041300093231F910F910C94EC1F0F931F930091E9
:1041400008031091090320910A0330910B036027A3
:104150007127822793271F910F910C94EC1F0895CC
:10416000292F220F920F990F890FA82FA695A69598
:10417000A695877051E001C0550F8A95EAF785E052
:10418000A89FD001112420E030E070E0F901EA0F8F
:10419000FB1FEF52FD4F4081CB01022E02C09695CE
:1041A00087950A94E2F78170992781958427852362
:1041B000842780832F5F3F4F2530310539F70895DD
:1041C000292F220F920F990F890F682F66956695F8
:1041D0006695982F977085E0689FB001112440E0A4
:1041E00050E080E0FA01E60FF71FEF52FD4F20810B
:1041F00030E0092E02C0369527950A94E2F7217027
:104200003327042E01C0220F0A94EAF7822B4F5F56
:104210005F4F4530510531F70895CF92DF92EF920D
:10422000FF920F931F93CF93DF938C01C0900C03E9
:10423000D0900D03E0900E03F0900F0380910803DF
:1042400090910903A0910A03B0910B03C82AD92ABF
:10425000EA2AFB2ACFE1D0E0D701C6010C2E04C028
:10426000B695A795979587950A94D2F780FF06C0D3
:10427000B8018C2F0E94160B019721F4219760F74B
:1042800080E001C08C2FDF91CF911F910F91FF90A3
:10429000EF90DF90CF900895CF93DF93EC010E94D1
:1042A0000D21BE010E94160BDF91CF9108951F933F
:1042B000CF93DF93EB0190919602992321F0CB01EC
:1042C0000E944C2113C0882349F0CB010E940D218C
:1042D000182F682FCE010E94B02004C0CB010E948D
:1042E000E020182FBE01812F0E94160BDF91CF9185
:1042F0001F91089580911003859585958595089562
:10430000809110038770089598E0899F900111248F
:10431000262B209310030C941220209110038095DB
:10432000822380931003982F977069F430E0482F10
:10433000082E000C550B2417350729F08595859517
:1043400085950C943320089590911003977081E027
:1043500009F480E00895E0910F01F091100180913F
:1043600034038083E0910F01F091100190818091DE
:104370003303892B8083E0910F01F091100190812C
:1043800080913203892B808380911103882381F0EF
:10439000E0910F01F09110019081892B8083809131
:1043A0000F01909110010E94E422811110921103DB
:1043B00080910F01909110010C94C61580913403E7
:1043C000089590913403892B809334030895809548
:1043D0009091340389238093340308951092340319
:1043E000089590913303892B80933303089580952A
:1043F00090913303892380933303089510923303FC
:10440000089590913203892B80933203089580950B
:1044100090913203892380933203089510923203DE
:1044200008958093110308951092110308958091C7
:1044300011030895CF92DF92EF92FF926C01EE2468
:10444000FF24C114D104E104F10421F0C701B60135
:1044500020E101C020E0C72ED82EE92EFF24C11490
:10446000D104E104F10419F0285FC701B6016B0122
:104470007C0154E0F694E794D794C7945A95D1F709
:10448000C114D104E104F10419F02C5FC701B60195
:104490006B017C0142E0F694E794D794C7944A9567
:1044A000D1F7C114D104E104F10419F02E5FC70162
:1044B000B601DC01CB01B695A79597958795892B19
:1044C0008A2B8B2B09F02F5F822FFF90EF90DF90CC
:1044D000CF90089580E090E00E94993321E08D3ED6
:1044E0009E4F09F020E0822F089580E090E00E9426
:1044F000993321E0019609F020E0822F089582E0AF
:1045000090E00C948B3383E090E00C948B3384E048
:1045100090E00C948B33682F84E090E00C949F33F0
:10452000AB01BC018FE090E00C94B133AB01BC0156
:1045300083E190E00C94B13360E070E0CB010C9427
:10454000962260E070E0CB010E9490220C949C22A5
:104550006DEE7EEF80E090E00E94BD3360E082E08F
:1045600090E00E949F3360E083E090E00E949F33E0
:1045700010920C0310920D0310920E0310920F0371
:1045800060E084E090E00E949F3360E085E090E08E
:104590000E949F3360E086E090E00E949F336FEFBF
:1045A00087E090E00E949F3340E050E0BA0188E04D
:1045B00090E00E94B13360E08DE090E00E949F3374
:1045C0000C94A1220C94A822FC0131969C01205E3F
:1045D0003F4F80E0919191118F5FE217F307D1F780
:1045E00008959C01FC0132969FEF80E041914617AF
:1045F00089F09F3F19F4411101C0982F8F5F8E31D0
:10460000A9F79F3F39F0F901E90FF11D97FDFA95E0
:10461000628308950895FC013296809620812613C6
:1046200001C010823196E817F907C1F70895262FC7
:104630002695269526952F3168F4FC01E20FF11D91
:10464000677021E030E001C0220F6A95EAF78181AE
:10465000282B21830895262F2695269526952F31E0
:1046600070F4FC01E20FF11D677021E030E001C041
:10467000220F6A95EAF720958181282321830895E6
:1046800020912001222329F02091AE0327FD0C94D4
:1046900017230C94F12220912001222329F020914C
:1046A000AE0327FD0C942B230C940B23FC013196B5
:1046B00080961192E817F907E1F7089508950C9490
:1046C0005E230E945F238091B403843049F11092ED
:1046D000360320E488E190E00FB6F894A895809323
:1046E00060000FBE2093600080E00E9437080E94A7
:1046F0005F2383B7817F846083BF83B7816083BF7B
:104700007894889583B78E7F83BF0FB6F894A89569
:1047100080916000886180936000109260000FBEFD
:1047200008950895CF930E94DB040E942B050E94F8
:104730009123C0E08C2F0E949905811104C0CF5FA6
:10474000CE30C1F701C081E0CF91089508950C9457
:10475000A6230E94DA1B0E94BA150E9437080C9407
:10476000A7231F920F920FB60F9211248F939F933E
:10477000AF93BF9380913603811113C08091AA0338
:104780009091AB03A091AC03B091AD034196A11DF4
:10479000B11D8093AA039093AB03A093AC03B09395
:1047A000AD03BF91AF919F918F910F900FBE0F906E
:1047B0001F90189582E084BD93E095BD9AEF97BD58
:1047C00080936E0008952FB7F8948091AA0390917A
:1047D000AB03A091AC03B091AD032FBF0895CF926E
:1047E000DF92EF92FF920F931F932FB7F8944091AF
:1047F000AA035091AB036091AC037091AD032FBF3E
:104800006A017B01EE24FF248C0120E030E0C01619
:10481000D106E206F30610F4415051099A01281B13
:10482000390BC9011F910F91FF90EF90DF90CF904E
:10483000089578941F920F920FB60F9211248F93C0
:104840009F93AF93BF938091AA039091AB03A091E4
:10485000AC03B091AD030196A11DB11D8093AA03D5
:104860009093AB03A093AC03B093AD03BF91AF9112
:104870009F918F910F900FBE0F901F901895F894F5
:1048800081E08093E00080E28093D800E9ECF0E0E2
:1048900010828FE19EE40197F1F700C000001DBA7D
:1048A000109268001CBC10BE1FBA10927A001092C1
:1048B0006E0010926F0010927100109272001082C0
:1048C000ECEBF0E0108214B817B81AB81DB810BAA3
:1048D000108215B818B81BB81EB811BA0C94003F56
:1048E00008950E946A22811102C00E94E2220E9461
:1048F0007F22809335030E94872290E09093AF033C
:104900008093AE030E948322682F70E080E090E0E5
:104910000C94B21F80913A0380FF0BC06091140188
:1049200085E0689FB0011124759567957595679529
:104930002BC081FF09C06091140185E0689FB00120
:1049400011247595679520C082FF07C060911401FE
:1049500085E0689FB001112417C090913B03992313
:10496000D1F060911301961788F72091140185E02A
:10497000289F90011124929FA001939F500D112414
:1049800070E0CA010E9464336038710540F461151B
:10499000710539F002C065E070E0862F08958FE759
:1049A000089581E0089580913A0380FF08C06091E6
:1049B000120170E0759567957595679521C081FF27
:1049C00006C06091120170E07595679519C082FF6D
:1049D00004C06091120170E010C090913B039923D4
:1049E000C1F0609111019617A0F780911201899F83
:1049F000C001112470E00E9464336038710528F40E
:104A00006115710521F0862F08958FE7089581E0E3
:104A1000089561E070E0F4CF803F21F40E948A2481
:104A2000819504C0813F29F40E948A2480933E032B
:104A30000895823F21F40E948A24819504C0833F17
:104A400029F40E948A2480933D030895893F19F434
:104A50000E94D32405C08A3F31F40E94D32481955B
:104A600080933F0308958B3F21F40E94D3248195C6
:104A700004C08C3F29F40E94D324809340030895FE
:104A8000843F21F480913C03816017C0853F21F46D
:104A900080913C03826011C0863F21F480913C03E9
:104AA00084600BC0873F21F480913C03886005C07F
:104AB000883F31F480913C03806180933C030895EA
:104AC0008D3F21F480913A0381600BC08E3F21F429
:104AD00080913A03826005C08F3F29F480913A03A8
:104AE000846080933A030895803F39F480913E03B7
:104AF00087FF6CC010923E0369C0813F29F480910A
:104B00003E031816BCF362C090913D03823F29F426
:104B100097FF5CC010923D0359C0833F19F41916EA
:104B2000CCF354C0893F41F480913F0318160CF038
:104B30004DC010923F034AC08A3F29F480913F0341
:104B400087FF44C0F6CF8B3F39F48091400387FF45
:104B50003DC0109240033AC08C3F29F4809140033D
:104B60001816BCF333C0843F21F480913C038E7F40
:104B700017C0853F21F480913C038D7F11C0863F93
:104B800021F480913C038B7F0BC0873F21F48091FF
:104B90003C03877F05C0883F31F480913C038F7EC2
:104BA00080933C0313C08D3F21F480913A038E7FA4
:104BB0000BC08E3F21F480913A038D7F05C08F3F5B
:104BC00029F480913A038B7F80933A0380913D03CF
:104BD00081110EC080913E0381110AC080913F0374
:104BE000811106C080914003811102C010923B03E5
:104BF00008958CE393E00E94D1150E94E3239093E3
:104C000038038093370308951F93CF93DF938091E8
:104C10003703909138030E94EF23AC0190913B033E
:104C2000992321F02091150130E006C0209139032D
:104C30008AE0289F900111244217530708F47BC093
:104C400080913D03C0913E03D0913F0310914003FA
:104C5000811107C0C1116BC0D11169C0111167C0AA
:104C60006AC09F3F19F09F5F90933B03181624F48E
:104C70000E948A2480933D0380913D0387FF05C0F5
:104C80000E948A24819580933D031C1624F40E947F
:104C90008A2480933E0380913E0387FF05C00E94D3
:104CA0008A24819580933E0330913D033323E1F0C4
:104CB00020913E032223C1F045EB3403C0011124AF
:104CC000892F990F990B009709F481E080933D0398
:104CD00035EB2303C0011124892F990F990B0097FD
:104CE00009F481E080933E031D1624F40E94D3242E
:104CF00080933F0380913F0387FF05C00E94D32428
:104D0000819580933F03111624F40E94D32480934D
:104D100040038091400387FF05C00E94D324819502
:104D200080934003DF91CF911F910C94F9259F3F11
:104D300009F099CFA1CFDF91CF911F910895ECE3B6
:104D4000F3E085E0DF011D928A95E9F710923B03BD
:104D500010923A030895833081F128F4813059F09C
:104D60008230D1F00895853009F449C0B8F1863019
:104D700009F456C0089580913903262F30E0280F9A
:104D8000311D2F3F310524F4680F609339030895D6
:104D90008FEF80933903089580911501262F30E01D
:104DA000280F311D2F3F310524F4680F6093150142
:104DB00008958FEF80931501089580911401262F97
:104DC00030E0280F311D2F3F310524F4680F609328
:104DD000140108958FEF80931401089580911301B9
:104DE000262F30E0280F311D2F3F310524F4680FA6
:104DF0006093130108958FEF8093130108958091BC
:104E00001201262F30E0280F311D2F3F310524F4E9
:104E1000680F6093120108958FEF80931201089537
:104E200080911101262F30E0280F311D2F3F3105D1
:104E300024F4680F6093110108958FEF809311019E
:104E40000895833011F128F4813049F0823091F0D7
:104E50000895853081F120F18630C1F10895809167
:104E60003903681720F4861B809339030895109244
:104E70003903089580911501681720F4861B8093EB
:104E80001501089510921501089580911401681775
:104E900020F4861B80931401089510921401089544
:104EA00080911301681720F4861B809313010895E5
:104EB00010921301089580911201681720F4861B47
:104EC00080931201089510921201089580911101AA
:104ED000681720F4861B8093110108951092110128
:104EE00008950F931F93873208F04DC08E3108F05C
:104EF00093C0803109F47DC008F5873009F46BC098
:104F000068F4863009F0A3C080913503817F8E7FDD
:104F10008093350381E0809342039AC08B3009F47B
:104F20008FC08E3009F093C08091350382FB222719
:104F300020F991E0922790FB82F964C0863109F450
:104F40007FC088F4813109F082C00E94DA1B809111
:104F5000AE0387FB222720F991E0922790FB87F987
:104F60008093AE036DC0893109F46AC08B3109F0BA
:104F70006EC08091350381FB222720F991E09227B2
:104F800090FB81F93FC0883309F45AC050F489324C
:104F900009F458C0853309F455C0873209F452C06A
:104FA00056C0833409F44EC028F48A3308F44FC045
:104FB000895333C0883409F04AC00E94DA1B0FEFCE
:104FC00013ED20E3015010402040E1F700C0000045
:104FD0000E943F2435C080913503982F90959170A1
:104FE00090FB80F98093350391112AC0897F877FD8
:104FF00010C08091350383FB222720F991E092278E
:1050000090FB83F9809335039923D1F08091350388
:1050100081608093350314C08D5141E050E060E021
:1050200070E08A019B0104C0000F111F221F331F73
:105030008A95D2F7C901B8010E94B21F0E94DA1BFB
:1050400081E006C061E070E080E090E0F5CF80E0B4
:105050001F910F91089580E0089580E008958E518A
:105060008A3030F4E82FF0E0E753FE4F8081089556
:1050700080E00895CF93C82F80914203813079F06A
:1050800018F08230E9F185C0E0910F01F091100134
:105090008081813169F0823209F07DC009C0E091E0
:1050A0000F01F09110018081813111F0823261F4A1
:1050B0008C2F0E942B28811104C08C2F0E947127F5
:1050C0001DC081E090E01AC08C2F0E942D28811114
:1050D00014C0C43179F048F4CB3079F0C03109F014
:1050E0005EC082E08093420308C0C93219F0C83321
:1050F00021F055C01092420352C081E0817051C02E
:10510000C93279F108F5C43161F1A0F4C73009F072
:1051100044C01092390384E180931501C0931401B7
:105120008CE38093130188E08093120188E28093DE
:10513000110133C082EE8C0F863078F58C2F0E94DF
:105140002F288093410329C0CE34E9F020F4CB34DA
:1051500021F56AE013C0C13579F0C235F1F461E0A0
:105160000DC080914103882319F01092410315C0AE
:1051700081E08093420315C061E006C08091410345
:105180000E94AB260AC06AE0809141030E94212759
:1051900004C01092420380E004C081E002C080E0BD
:1051A000ADCFCF9108958091630308950F931F931E
:1051B000CF93DF9300D01F92CDB7DEB78C010E9452
:1051C0004E2B823011F0843019F593E099831B83C4
:1051D0000A839093E9008FEF9091E800815095FD4C
:1051E00006C095ED9A95F1F700008111F5CF8091F9
:1051F000E80085FF0DC040E050E063E070E0CE01C4
:1052000001960E946B2B8091E8008E778093E800D6
:105210000F900F900F90DF91CF911F910F910895F4
:10522000CF93DF9300D01F92CDB7DEB72091B403A8
:10523000243031F522E02983805891099B838A83A9
:1052400083E08093E9008FEF9091E800815095FD15
:1052500006C095ED9A95F1F700008111F5CF809188
:10526000E80085FF0DC040E050E063E070E0CE0153
:1052700001960E946B2B8091E8008E778093E80066
:105280000F900F900F90DF91CF910895CF93DF9300
:10529000EC010E944E2B823011F08430F9F482E050
:1052A0008093E9009FEF8091E800915085FD06C052
:1052B00085ED8A95F1F700009111F5CF8091E80016
:1052C00085FF0CC040E050E065E070E0CE010E9438
:1052D0006B2B8091E8008E778093E800DF91CF916F
:1052E0000895CF93DF93EC010E944E2B823019F08A
:1052F000843009F047C0809120018823E1F080913B
:10530000AE0387FF18C084E08093E9008FEF90918F
:10531000E800815095FD06C095E19A95F1F70000EF
:105320008111F5CF8091E80085FF2CC040E050E06E
:1053300060E270E017C081E08093E9008FEF909108
:10534000E800815095FD06C095ED9A95F1F70000B3
:105350008111F5CF8091E80085FF14C040E050E056
:1053600068E070E0CE010E946B2B8091E8008E77A0
:105370008093E80080E2FE01A3E4B3E001900D9287
:105380008A95E1F7DF91CF9108958091B303811160
:1053900009C00E94002D0E945D2D8091E200846072
:1053A0008093E20008951092B3030895089508953C
:1053B0000C94A92342E061EC81E00E947A2C42E047
:1053C00061EC82E00E947A2C42E061EC83E00E9472
:1053D0007A2C42E261EC84E00C947A2C8091B60342
:1053E000833009F455C030F4813071F0823009F413
:1053F0008EC008958A3009F47AC08B3009F460C0F9
:10540000893009F09CC020C08091B503813A09F031
:1054100096C08091E800877F8093E8008091B9036F
:105420009091BA03892B21F460E283E493E003C0F6
:1054300060E080E090E070E00E94B62B8091E80090
:105440008B778093E80008958091B503813209F04D
:1054500076C08091B9039091BA03009719F0039731
:1054600009F06DC08091E800877F8093E80080910B
:10547000E80082FD05C08091B4038111F8CF5FC0C0
:105480008091F100809363038091E8008B7753C093
:105490008091B503813A09F052C08091B90390918F
:1054A000BA03892B09F04BC08091E800877F809375
:1054B000E8008091E80080FFFCCF8091200136C099
:1054C0008091B5038132D9F58091B9039091BA03E7
:1054D000892BA9F58091E800877F8093E8000E94DE
:1054E000AF2C8091B703809320010C94DA1B80913C
:1054F000B503813221F58091E800877F8093E80031
:105500000E94AF2C8091B80380936403089580912A
:10551000B503813AA1F48091E800877F8093E80089
:105520008091E80080FFFCCF809164038093F100BC
:105530008091E8008E778093E8000C94AF2C08955A
:1055400084B7877F84BF0FB6F894A89580916000D8
:10555000886180936000109260000FBE80E88093A5
:105560006100109261000E9409160E94002D0E94A5
:105570005D2D8091E20084608093E20078940E9427
:10558000EC2F0E940D1686E191E00E94B5158091E6
:10559000B403853069F40E9461238091B2038823AB
:1055A000B1F30E949223882391F30E94552BEFCFF1
:1055B0000E941B160E94AF14EACF0C94DF2A292FF9
:1055C000332723303105C9F064F42130310581F0EF
:1055D0002230310509F049C08DE690E028E336E03D
:1055E00048C02132310521F12232310571F13DC02F
:1055F00082E190E025EA36E03CC0992781309105B0
:1056000071F02CF4892B89F5E4E3F6E00DC08230CB
:10561000910541F0039749F5EEEFF5E005C0ECE1A7
:10562000F6E002C0E4E0F6E0849190E09F0121C042
:1056300064307105D0F4660F771FFB01E152FE4F15
:105640002081318189E090E014C06430710568F4F4
:10565000FB01EE0FFF1FE952FE4F20813181FB015C
:10566000ED52FE4F808190E004C080E090E020E0A9
:1056700030E0FA013183208308950895CF93C82F35
:105680000E943D2BC0936503CF9108958091B40390
:10569000843011F081E0089582E0089580916503DF
:1056A000811102C00C94462B089580E189BD82E1EE
:1056B00089BD09B400FEFDCF8091D8008F7D809315
:1056C000D8008091E00082608093E0008091E0004B
:1056D00081FDFCCF0895CF92DF92EF92FF920F935E
:1056E0001F93CF93DF93EC018B016A010E94CE2CB4
:1056F000811133C0C114D10439F0F6018081918148
:10570000081B190BC80FD91FE12CF12C011511052D
:1057100019F18091E80085FD16C08091E8008E7730
:105720008093E800C114D10449F0F6018081918191
:10573000E80EF91EF182E08285E00FC00E94CE2CB7
:10574000882321F30AC089918093F1000150110947
:10575000FFEFEF1AFF0ADACF80E0DF91CF911F91C0
:105760000F91FF90EF90DF90CF9008952091BB03B1
:105770003091BC032617370748F06115710539F4DD
:105780002091E8002E772093E80001C0B90140E0A5
:1057900061157105A9F12091B403222309F443C0D6
:1057A000253009F442C02091E80023FD40C020913B
:1057B000E80022FD32C02091E80020FFE9CF4091AF
:1057C000F3002091F20030E0342BFC01CF01611591
:1057D000710559F02830310540F481918093F10032
:1057E000615071092F5F3F4FF1CF41E02830310503
:1057F00009F040E02091E8002E772093E800C8CF20
:105800004111C9CF0AC08091B403882361F085306B
:1058100061F08091E80083FD0AC08091E80082FF7A
:10582000F2CF80E0089582E0089583E0089581E05A
:1058300008952091BB033091BC032617370748F029
:105840006115710539F42091E8002E772093E80066
:1058500001C0B901FC0120E06115710591F1809151
:10586000B403882309F440C0853009F43FC0809117
:10587000E80083FD3DC08091E80082FD2FC080914B
:10588000E80080FFE9CF2091F3008091F20090E0E2
:10589000922B6115710559F08830910540F42491DF
:1058A0002093F1003196615071090196F2CF21E009
:1058B000089709F020E08091E8008E778093E80057
:1058C000CBCF2111CCCF0AC08091B403882361F0E3
:1058D000853061F08091E80083FD0AC08091E80086
:1058E00082FFF2CF80E0089582E0089583E008957A
:1058F00081E00895982F973058F59093E900981714
:1059000039F07091EC002091ED005091F00003C04F
:10591000242F762F50E021FF19C03091EB003E7FFD
:105920003093EB003091ED003D7F3093ED003091EE
:10593000EB0031603093EB007093EC002093ED00AE
:105940005093F0002091EE0027FF07C09F5FD3CF58
:105950008F708093E90081E0089580E00895809140
:10596000B50387FF11C08091E80082FD05C08091DA
:10597000B4038111F8CF11C08091E8008B770BC080
:105980008091B403882349F08091E80080FFF8CF2C
:105990008091E8008E778093E80008952091E400DC
:1059A0003091E50095E64091EC00842F817040FF36
:1059B00022C08091E80080FD1CC08091B403882340
:1059C00091F0853091F08091EB0085FD10C0409101
:1059D000E4005091E5004217530729F39A019150D2
:1059E00011F784E0089582E0089583E0089581E04E
:1059F000089580E008954091E80042FFDECF0895C9
:105A00000E946E2D0E94762DE0EEF0E08081816094
:105A10008083E8EDF0E080818F77808319BCA7ED6B
:105A2000B0E08C918E7F8C9380818F7E80831092EA
:105A3000B30308950F931F93CF93DF930E946E2DAE
:105A40000E94762DC8EDD0E088818F778883888189
:105A50008068888388818F7D888319BC1092B40305
:105A60001092B0031092B2031092B10300EE10E056
:105A7000F80180818B7F808388818160888342E008
:105A800060E080E00E947A2CE1EEF0E080818E7F81
:105A90008083E2EEF0E08081816080838081886095
:105AA0008083F80180818E7F8083888180618883F4
:105AB000DF91CF911F910F910895E8EDF0E0808183
:105AC0008F7E8083E7EDF0E080818160808384E0D9
:105AD00082BF81E08093B3030C941A2DE8EDF0E0CF
:105AE00080818E7F80831092E20008951092DA0008
:105AF0001092E10008951F920F920FB60F92112499
:105B00002F933F934F935F936F937F938F939F93C5
:105B1000AF93BF93EF93FF938091E10082FF0BC09F
:105B20008091E20082FF07C08091E1008B7F80932B
:105B3000E1000E94EB2F8091DA0080FF1FC080916E
:105B4000D80080FF1BC08091DA008E7F8093DA003E
:105B50008091D90080FF0DC080E189BD82E189BDBF
:105B600009B400FEFDCF81E08093B4030E94C529F3
:105B700005C019BC1092B4030E94D3298091E100A2
:105B800080FF19C08091E20080FF15C08091E20083
:105B90008E7F8093E2008091E20080618093E2003A
:105BA0008091D80080628093D80019BC85E08093F2
:105BB000B4030E94D7298091E10084FF30C0809116
:105BC000E20084FF2CC080E189BD82E189BD09B477
:105BD00000FEFDCF8091D8008F7D8093D80080910A
:105BE000E1008F7E8093E1008091E2008F7E8093C0
:105BF000E2008091E20081608093E2008091B00336
:105C0000882311F084E007C08091E30087FD02C083
:105C100081E001C083E08093B4030E94D829809181
:105C2000E10083FF29C08091E20083FF25C08091BD
:105C3000E100877F8093E10082E08093B4031092BB
:105C4000B0038091E1008E7F8093E1008091E200BB
:105C50008E7F8093E2008091E20080618093E20079
:105C600042E060E080E00E947A2C8091F000886041
:105C70008093F0000E94D629FF91EF91BF91AF91E0
:105C80009F918F917F916F915F914F913F912F9154
:105C90000F900FBE0F901F9018951F920F920FB686
:105CA0000F9211242F933F934F935F936F937F93A2
:105CB0008F939F93AF93BF93CF93DF93EF93FF9314
:105CC000C091E900CF708091EC00D82FD17080FD99
:105CD000D0E81092E9008091F000877F8093F00077
:105CE00078940E94912E1092E9008091F0008860D3
:105CF0008093F000CD2BCF70C093E900FF91EF911E
:105D0000DF91CF91BF91AF919F918F917F916F91D3
:105D10005F914F913F912F910F900FBE0F901F9069
:105D200018951F93CF93DF93CDB7DEB7AA970FB621
:105D3000F894DEBF0FBECDBFE5EBF3E088E08E0F39
:105D40009091F10091938E13FBCF0E94EE298091E8
:105D5000E80083FF28C18091B5039091B603492FD5
:105D600050E04A30510508F01EC1FA01E755FF4FD7
:105D70000C947833803821F0823809F014C108C0BF
:105D80008091B1039091B203992389F082600FC092
:105D90008091B9038F70873008F005C18093E900C6
:105DA0008091EB0085FB882780F91092E9009091A3
:105DB000E800977F9093E8008093F1001092F10043
:105DC000D0C0282F2D7F09F0EEC0882319F0823033
:105DD00061F0E9C08091B703813009F0E4C09330ED
:105DE00009F080E08093B2032EC08091B703811147
:105DF0002AC08091B9038F702FEF280F263008F04A
:105E0000D2C08093E9002091EB0020FF1CC09330AA
:105E100021F48091EB00806214C09091EB009061BE
:105E20009093EB0021E030E0A90102C0440F551F20
:105E30008A95E2F74093EA001092EA008091EB0025
:105E400088608093EB001092E9008091E800877FE2
:105E50008093E8000E94AF2CA6C08111A4C01091CD
:105E6000B7031F778091E3008078812B8093E30054
:105E70008091E800877F8093E8000E94AF2C80919A
:105E8000E80080FFFCCF8091E30080688093E3000E
:105E9000111102C082E001C083E08093B40383C08B
:105EA0008058823008F07FC08091B7039091B8038A
:105EB0008C3D53E0950779F583E08A838AE28983F4
:105EC0004FB7F894DE01139620E03EE051E2E32F55
:105ED000F0E050935700E49120FF03C0E295EF708B
:105EE0003F5FEF708E2F90E0EA3010F0C79601C050
:105EF000C0968D939D932F5F243149F74FBF8091BA
:105F0000E800877F8093E8006AE270E0CE010196A6
:105F10000E94B62B15C06091B9037091BA03AE010F
:105F20004F5F5F4F0E94DD2ABC01892BE1F1909108
:105F3000E800977F9093E80089819A810E94192C4C
:105F40008091E8008B778093E8002DC0803859F568
:105F50008091E800877F8093E8008091B003809370
:105F6000F1008091E8008E7773CF81111CC0909171
:105F7000B7039230C0F48091E800877F8093E800F7
:105F80009093B0030E94AF2C8091B003811106C0A2
:105F90008091E30087FD02C081E001C084E080932E
:105FA000B4030E94DA298091E80083FF0AC080913F
:105FB000E800877F8093E8008091EB008062809307
:105FC000EB00AA960FB6F894DEBF0FBECDBFDF91EF
:105FD000CF911F9108950895CF938091B4038823A2
:105FE000A1F0C091E900CF709091EC00892F8170F1
:105FF00090FD80E8C82B1092E9008091E80083FDB5
:106000000E94912ECF70C093E900CF91089550580F
:10601000BB27AA270E941F300C94CA310E94BC31B2
:1060200038F00E94C33120F039F49F3F19F426F470
:106030000C9492310EF4E095E7FB0C948C31E92F2F
:106040000E94DB3158F3BA1762077307840795077C
:1060500020F079F4A6F50C94FD310EF4E0950B2EAA
:10606000BA2FA02D0B01B90190010C01CA01A001AA
:106070001124FF27591B99F0593F50F4503E68F105
:106080001A16F040A22F232F342F4427585FF3CF46
:10609000469537952795A795F0405395C9F77EF417
:1060A0001F16BA0B620B730B840BBAF09150A1F060
:1060B000FF0FBB1F661F771F881FC2F70EC0BA0FE6
:1060C000621F731F841F48F4879577956795B7956E
:1060D000F7959E3F08F0B0CF9395880F08F0992769
:1060E000EE0F9795879508950E9488300C94CA31D9
:1060F0000E94C33158F00E94BC3140F029F45F3F48
:1061000029F00C948C3151110C94FE310C94923185
:106110000E94DB3168F39923B1F3552391F3951B6A
:10612000550BBB27AA2762177307840738F09F5FB8
:106130005F4F220F331F441FAA1FA9F335D00E2E25
:106140003AF0E0E832D091505040E695001CCAF792
:106150002BD0FE2F29D0660F771F881FBB1F261755
:1061600037074807AB07B0E809F0BB0B802DBF012C
:10617000FF2793585F4F3AF09E3F510578F00C94FB
:106180008C310C94FE315F3FE4F3983ED4F3869556
:1061900077956795B795F7959F5FC9F7880F911D1C
:1061A0009695879597F90895E1E0660F771F881F08
:1061B000BB1F621773078407BA0720F0621B730BBB
:1061C000840BBA0BEE1F88F7E095089529F416F0BA
:1061D0000C948C310C94FD310C9492310E94E3317B
:1061E000A8F39638A0F707F80F92E8942BE33AEA61
:1061F00048EB5FE70E9490320F920F920F924DB7DB
:106200005EB70F920E944632E6E6F1E00E949531B9
:106210004F915F91EF91FF91E595EE1FFF1F49F0C0
:10622000FE57E0684427EE0F441FFA95E1F74195C9
:10623000550B0E9410320F9007FE0C940432089503
:106240000E94E33188F09F5798F0B92F9927B751F2
:10625000B0F0E1F0660F771F881F991F1AF0BA950A
:10626000C9F714C0B13091F00E94FD31B1E008953A
:106270000C94FD31672F782F8827B85F39F0B93F2C
:10628000CCF3869577956795B395D9F73EF49095BD
:106290008095709561957F4F8F4F9F4F0895E8943B
:1062A00009C097FB3EF490958095709561957F4F5E
:1062B0008F4F9F4F9923A9F0F92F96E9BB2793950C
:1062C000F695879577956795B795F111F8CFFAF41C
:1062D000BB0F11F460FF1BC06F5F7F4F8F4F9F4F4D
:1062E00016C0882311F096E911C0772321F09EE8AB
:1062F000872F762F05C0662371F096E8862F70E011
:1063000060E02AF09A95660F771F881FDAF7880FEA
:106310009695879597F9089597F99F6780E870E0BB
:1063200060E008959FEF80EC0895DF93CF931F9373
:106330000F93FF92EF92DF927B018C01689406C06D
:10634000DA2EEF010E948D32FE01E894A59125918D
:10635000359145915591A6F3EF010E941F30FE0142
:106360009701A801DA9469F7DF90EF90FF900F9101
:106370001F91CF91DF91089500240A9416161706F5
:1063800018060906089500240A9412161306140626
:1063900005060895092E0394000C11F4882352F089
:1063A000BB0F40F4BF2B11F460FF04C06F5F7F4F41
:1063B0008F4F9F4F089557FD9058440F551F59F028
:1063C0005F3F71F04795880F97FB991F61F09F3FE2
:1063D00079F087950895121613061406551FF2CF0B
:1063E0004695F1DF08C0161617061806991FF1CF5B
:1063F00086957105610508940895E894BB27662782
:106400007727CB0197F908959B01AC0160E070E01C
:1064100080E89FE30C9474300C948C310C94EF3230
:106420000E94E331D8F39923C9F3940F511DA3F3CC
:106430009150504094F059F0882332F0660F771F46
:10644000881F91505040C1F79E3F51052CF7880F8F
:10645000911D9695879597F908955F3FACF0983E0A
:106460009CF0BB27869577956795B79508F4B16042
:106470009395C1F7BB0F58F711F460FFE8CF6F5F3A
:106480007F4F8F4F9F4FE3CF0C94FE31FA01DC0119
:10649000AA0FBB1F9B01AC01BF5728F4222733274B
:1064A0004427507820C0B75190F4AB2F0024469574
:1064B00037952795011CA395D2F3002071F0220F88
:1064C000331F441FB395DAF30ED00C9407306130BC
:1064D0007105A0E88A07B94630F49B01AC01662734
:1064E000772788279078309621F020833183428364
:1064F000538308950E948D320C94CA310E94BC319E
:1065000038F00E94C33120F0952311F00C948C31A7
:106510000C94923111240C94FE310E94DB3170F303
:10652000959FC1F3950F50E0551F629FF001729F38
:10653000BB27F00DB11D639FAA27F00DB11DAA1F47
:10654000649F6627B00DA11D661F829F2227B00D94
:10655000A11D621F739FB00DA11D621F839FA00D1F
:10656000611D221F749F3327A00D611D231F849F6F
:10657000600D211D822F762F6A2F11249F575040C6
:106580009AF0F1F088234AF0EE0FFF1FBB1F661F41
:10659000771F881F91505040A9F79E3F510580F00A
:1065A0000C948C310C94FE315F3FE4F3983ED4F3AD
:1065B000869577956795B795F795E7959F5FC1F7AE
:1065C000FE2B880F911D9695879597F908959F93B7
:1065D0000E94FF320F9007FCEE5F0C9428339F3F20
:1065E00031F0915020F4879577956795B795880F8E
:1065F000911D9695879597F908950C9492310E9474
:10660000E331D8F3E894E0E0BB279F57F0F02AEDA0
:106610003FE049EC06C0EE0FBB0F661F771F881FD7
:1066200028F0B23A62077307840728F0B25A620B67
:10663000730B840BE3959A9572F7803830F49A9532
:10664000BB0F661F771F881FD2F790480C94F1325A
:10665000EF93E0FF07C0A2EA2AED3FE049EC5FEBD1
:106660000E941F300E94CA310F90039401FC905881
:10667000EEE8F1E00C943C339F938F937F936F93FC
:10668000FF93EF939B01AC010E947A32EF91FF914F
:106690000E9495312F913F914F915F910C947A32E6
:1066A000AA1BBB1B51E107C0AA1FBB1FA617B70738
:1066B00010F0A61BB70B881F991F5A95A9F7809554
:1066C0009095BC01CD01089597FB072E16F4009418
:1066D00007D077FD09D00E94503307FC05D03EF467
:1066E000909581959F4F0895709561957F4F08957E
:1066F000EE0FFF1F0590F491E02D0994FC0141502D
:10670000504030F001900616D1F73197CF0108952F
:10671000882799270895F999FECF92BD81BDF89AEF
:10672000992780B50895A6E1B0E044E050E00C94CC
:10673000C533A8E1B0E042E050E00C94C533262F09
:10674000F999FECF92BD81BDF89A019700B4021667
:1067500039F01FBA20BD0FB6F894FA9AF99A0FBE15
:1067600008950396272F0E94A0330E949F33252F60
:106770000E94A033242F0C94A0330196272F0E944F
:10678000A0330C949F33DC01CB01FC01F999FECFBF
:1067900006C0F2BDE1BDF89A319600B40D924150A9
:0A67A0005040B8F70895F894FFCFB9
:1067AA002000010201191A1B1C1D1E1F2021221282
:1067BA000328083C0714D328712946291029D6280A
:1067CA0001000D010D020D030D040D050D000C0154
:1067DA000C020C030C040C050C000B010B020B033E
:1067EA000B040B050B000A010A020A030A040A0534
:1067FA000A00090109020903090409050900080137
:10680A00080208030804080508000701070207032D
:10681A000704070507000601060206030604060523
:10682A000600050105020503050405050500040126
:10683A00040204030404040504000301030203031D
:10684A000304030503000201020202030204020513
:10685A000200010101020103010401050100000116
:10686A0000020003000400050001020304050607F4
:10687A00080900404D363973072607F006B7064A5D
:08688A000663067C069506007A
:00000001FF
